S021000064656D6F70726F675F6F6C696D65785F73746D3332703130332E737265639D
S31508006000005000206D780008BD780008BD780008AB
S31508006010BD780008BD780008BD78000800000000BB
S31508006020000000000000000000000000BD78000825
S31508006030BD78000800000000BD780008F578000863
S31508006040BD780008BD780008BD780008BD7800084E
S31508006050BD780008BD780008BD780008BD7800083E
S31508006060BD780008BD780008BD780008BD7800082E
S31508006070BD780008BD780008BD780008BD7800081E
S31508006080BD780008BD780008BD780008BD7800080E
S31508006090BD780008BD780008BD780008BD780008FE
S315080060A0BD780008BD780008BD780008BD780008EE
S315080060B0BD780008BD780008BD780008BD780008DE
S315080060C0BD780008BD780008BD780008BD780008CE
S315080060D0BD780008BD780008BD780008BD780008BE
S315080060E0BD780008BD780008BD78000800000000EB
S315080060F00000000000000000000000000000000092
S3150800610000000000000000005FF808F1EE11AA5533
S3150800611010B5054C237833B9044B13B10448AFF3D3
S3150800612000800123237010BD0C0000200000000031
S315080061304879000808B5034B1BB103490348AFF378
S31508006140008008BD00000000100000204879000803
S3150800615008B50848084B03604FF4614343600023C1
S315080061608360C360036183610C224261C36101F0ED
S31508006170ACF908BD90000020004400402DE9F0412C
S3150800618004460D461746984601F074F8154BA3FBCE
S3150800619000308009002201E00132D2B2112A1ED84D
S315080061A0114B13F8121003EB420393F801E001EBCD
S315080061B00E0303FB0443B0FBF3FC03FB1C06002E93
S315080061C0EAD11FFA8CF32B80013B9BB2B3F5806FA3
S315080061D0E2D2397088F800E00120BDE8F08100209D
S315080061E0BDE8F081D34D62107479000870B58CB0A3
S315080061F00025ADF82E508DF82D500CAB03F8045D34
S315080062000DF12D020DF12E014FF4FA70FFF7B6FFCE
S315080062101D4C1E4E266025631D4B6363A561E56113
S3150800622025626562A562E562A560E5609DF82D3088
S31508006230013B1B0423619DF82C30013B1B05636160
S31508006240BDF82E306360204600F0C0F92368B342DB
S3150800625018D00E23069300230793012208924CF6C2
S31508006260E041019102934FF6E071039104210491F4
S31508006270059309920E230A936944034800F022F90C
S315080062800CB070BD0695E6E72800002000640040C3
S315080062906C00002008B5002301220146034801F0DE
S315080062A043F908B1002008BD012008BD9000002070
S315080062B008B5FFF74DFFFFF799FF08BDBFF34F8FEE
S315080062C00549CA6802F4E062044B1343CB60BFF386
S315080062D04F8F00BFFDE700BF00ED00E00400FA05A0
S315080062E008B5214B1B78B3B92048FFF7D3FF01281F
S315080062F000D008BD1D4B1B78013BDBB23F2BF8D8FD
S3150800630001F0F4FA1A4B18600122174B1A70002292
S31508006310184B1A7008BD174B1B78013313481844DD
S31508006320FFF7B8FF01280AD001F0E0FA104B1B6806
S3150800633064339842DDD900220B4B1A70D9E70D4A0F
S3150800634013780133DBB21370084A12789342D0D11E
S315080063500021054A1170054A5278FF2AC9D1022B35
S31508006360C7D1FFF7ABFF00BF11010020D000002006
S31508006370140100201201002008B5002211460E481B
S3150800638000F0C5F940B90C4B5B6B196840F26762BF
S31508006390914202D0002232B908BD9A680AB1002299
S315080063A0F9E70122F7E71A7DFF2AF5D11B69022BC7
S315080063B0F2D1FFF783FF00BF2800002008B5FFF7DA
S315080063C08FFFFFF7D9FF08BD08B501224FF48051AA
S315080063D0014800F04BFC08BD0010014010B501F063
S315080063E085FA104B1B68C31AB3F5FA7F0ED3044619
S315080063F00D4B1B785BB901220B4B1A7000224FF428
S3150800640080510A4800F032FC064B1C6010BD002281
S31508006410054B1A7001224FF48051044800F026FCFF
S31508006420F2E700BF1C0100201801002000100140FF
S3150800643010B504460E4B18784FF47A73B3FBF0F395
S315080064400C4A1068B0FBF3F000F0EEFA68B90F2CAE
S3150800645001D9012010BD002221464FF0FF3000F07F
S31508006460B1FA054B1C60002010BD012010BD00BF0D
S3150800647000000020080000200400002008B5074A94
S31508006480136843F010031360032000F089FA002014
S31508006490FFF7CEFF01F028F9002008BD00200240D2
S315080064A0034A1168034B1B780B441360704700BFFF
S315080064B02001002000000020014B1868704700BF2B
S315080064C020010020F0B44B6901229A400468D4F8F0
S315080064D0003223F47C534D6A43EA052343F0010353
S315080064E0C4F800320568D5F81C42D3431C40C5F8E9
S315080064F01C42CC69C4B90568D5F80C421C40C5F8DD
S315080065000C4206684C69CF688D8845EA07454834C9
S3150800651046F8345004684E698F680D8845EA074581
S31508006520483604EBC6046560CC69012C1ED08C691C
S31508006530002C35D10568D5F804421C40C5F804423C
S315080065400C69002C33D10468D4F814522B40C4F8D3
S3150800655014320B6A012B31D00268D2F8003223F0CC
S315080065600103C2F800320020F0BC70470568D5F870
S315080065700C421443C5F80C4206684C690F688D88AE
S3150800658045EA0745483446F8345004684E698F682A
S315080065908D8945EA0745483604EBC6046560C6E7B3
S315080065A00568D5F804421443C5F80442C8E70468E8
S315080065B0D4F814321343C4F81432CAE70368D3F87C
S315080065C01C120A43C3F81C22C6E77047002800F0CD
S315080065D09C8038B5044690F83C3003B3022384F80F
S315080065E03C302268136823F002031360226813689C
S315080065F043F001031360FFF75FFF054623685A68F7
S3150800660012F0010F10D1FFF757FF401B0A28F5D9E2
S31508006610032084F83C00002384F83D3038BD80F818
S315080066203D30FFF7D2FFD9E75A6812F0010F5DD067
S31508006630A269012A43D00022E169012941D022F04A
S315080066404002216A01293FD022F02002616A01290D
S315080066503DD022F01002A16A01293BD022F008029F
S31508006660E16A012939D022F00402196821F0FC01F7
S315080066700A431A602168A368E26813432269134330
S31508006680626913436268013A1343CB61226813684F
S3150800669023F001031360FFF70FFF054623685A68C6
S315080066A012F0010F1CD0FFF707FF401B0A28F5D987
S315080066B0032084F83C00002384F83D3038BD80224E
S315080066C0BAE742F04002BCE742F02002BEE742F0D9
S315080066D01002C0E742F00802C2E742F00402C4E72B
S315080066E05B6813F0010F08D0002300E0002333B9DC
S315080066F0042384F83C30012038BD0123F7E7002045
S315080067002064012384F83C3038BD01207047F8B571
S315080067100D46B9B990F83C30DBB2222B00F02F8138
S3150800672090F83C30DBB2422B00F02B8190F83C30DD
S31508006730DBB2622B00F0278190F83C30DBB2722B7B
S3150800674000F02381012D15D090F83D30012B00F083
S315080067502481012380F83D30B5BB90F83C30DBB28C
S31508006760322B29D0522B2BD0122B1CD0222380F867
S315080067703C301BE090F83C30DBB2322B00F007814E
S3150800678090F83C30DBB2522B00F0038190F83C3095
S31508006790DBB2622B00F0FF8090F83C30DBB2722B44
S315080067A0D2D10220F8BD422380F83C301646044672
S315080067B0FFF782FE074638E0622380F83C30F5E7AB
S315080067C0722380F83C30F1E790F83C30DBB2222B9C
S315080067D00BD0422B0DD0122B03D0322380F83C303D
S315080067E0E4E7522380F83C30E0E7622380F83C3047
S315080067F0DCE7722380F83C30D8E726B1FFF75CFE69
S31508006800C01B864211D2032084F83C00002384F87A
S315080068103D30F8BD23681B6913F0030F0CBF012335
S31508006820002363B1B6F1FF3FE7D1002DF2D123680B
S31508006830DB6813F0030F0CBF01230023F1E7002DDB
S3150800684067D1636B216805F11B0212018A5802F0B1
S3150800685004029A60002A5ED1216805F11B02120122
S315080068608A58520D1A60216805F11B0212018958CF
S3150800687001F00201D96021681144496801F00F014D
S31508006880196121680A445268C2F30722DA611D6257
S3150800689021682A011144D1F8B811197521681144E3
S315080068A0D1F8B811090A597521681144D1F8B811F7
S315080068B0090C997521681144D1F8B811090ED975D2
S315080068C021681144D1F8BC11197621681144D1F810
S315080068D0BC11090A597621681144D1F8BC11090C72
S315080068E0997621680A44D2F8BC21120EDA76D5B90F
S315080068F023682022DA604DBB94F83C30DBB2622B69
S315080069001CD0722B1ED0422B11D0012384F83C30A8
S3150800691010E0A36B96E7216805F11B0212018A585D
S31508006920D2085A609FE7236820221A61E3E71223F8
S3150800693084F83C30002084F83D00F8BD322384F802
S315080069403C30F7E7522384F83C30F3E794F83C30C0
S31508006950DBB2622B0BD0722B0DD0522B03D0012346
S3150800696084F83C30E6E7122384F83C30E2E7222339
S3150800697084F83C30DEE7422384F83C30DAE702202C
S31508006980F8BD0220F8BD0220F8BD0220F8BD02209D
S31508006990F8BD0220F8BD0220F8BD0220F8BD0000AF
S315080069A0074AD36823F4E0631B041B0C000200F4B7
S315080069B0E060184340F0BF6040F40030D060704794
S315080069C000ED00E030B4164BDB68C3F30223C3F1D5
S315080069D00704042C28BF04241D1D062D17D9033BC4
S315080069E0012505FA04F4013C2140994005FA03F310
S315080069F0013B1340194300280BDB0901C9B200F11A
S31508006A00604000F5614080F8001330BC70470023F1
S31508006A10E6E700F00F000901C9B2024B1954F4E782
S31508006A2000ED00E014ED00E00138B0F1807F0AD2F5
S31508006A30064B5860F021064A82F823100020986019
S31508006A4007221A6070470120704700BF10E000E077
S31508006A5000ED00E0042805D0054A136823F0040376
S31508006A6013607047024A136843F0040313607047C3
S31508006A7010E000E0704708B5FFF7FCFF08BD00000E
S31508006A80F0B583B00026344671E0002D00F0A180F1
S31508006A90012D00D1CE68FF2B00F2AF808646FF2B72
S31508006AA000F2AE80A500DEF800200F27AF4022EAEC
S31508006AB0070206FA05F52A43CEF800204A6812F0BE
S31508006AC0805F53D0634A956945F0010595619269DF
S31508006AD002F001020192019AA508AF1C5E4A52F81B
S31508006AE0272004F00307BF004FF00F0E0EFA07FE2B
S31508006AF022EA0E02DFF870E1704500F088800EF594
S31508006B00806E704500F086800EF5806E704500F048
S31508006B1084800EF5806E704576D04FF0040E0EFA1E
S31508006B2007F73A4302354C4F47F825204A6812F4CE
S31508006B30803F75D0494D2A681A432A604A6812F47C
S31508006B40003F73D0454D6A681A436A604A6812F472
S31508006B50801F71D0414DAA681A43AA604A6812F488
S31508006B60001F6FD03D4DEA681343EB6001340F2CCC
S31508006B706ED80122A2400B6813409A42F6D14D689E
S31508006B80122D30D00BD8022D2AD07FF67EAF032DDA
S31508006B902FD0112D7FF47FAFCE6804367BE7304FB8
S31508006BA0BD4216D00CD92F4FBD4212D007F58037FB
S31508006BB0BD420ED0A7F58017BD427FF46CAF08E042
S31508006BC0A7F58017BD4204D007F58037BD427FF48C
S31508006BD062AF8D687DB1012D08D0426108265AE75B
S31508006BE0CE68083657E7CE680C3654E702610826A1
S31508006BF051E700264FE704264DE700F1040E4EE75D
S31508006C00A4F10805AD004EE74FF0030E87E74FF0F5
S31508006C10000E84E74FF0010E81E74FF0020E7EE783
S31508006C200E4D2A6822EA03022A6087E70B4D6A6836
S31508006C3022EA03026A6089E7084DAA6822EA030283
S31508006C40AA608BE7054DEA6822EA0303EB608DE745
S31508006C5003B0F0BD001002400000014000040140EE
S31508006C6000002110000031100008014012B9090483
S31508006C70016170470161704782B0084B1B68084A7A
S31508006C80A2FB03235B0A00FB03F0019000BF019BF4
S31508006C905A1E0192002BF9D102B070470800002055
S31508006CA0D34D621070B582B00446036813F0010F25
S31508006CB03DD0AC4B5B6803F00C03042B2ED0A94BDC
S31508006CC05B6803F00C03082B23D06368B3F5803F99
S31508006CD051D0002B55D103F1804303F504331A68CC
S31508006CE022F480321A601A6822F480221A606368D5
S31508006CF0002B60D0FFF7E0FB05469A4B1B6813F4A0
S31508006D00003F14D1FFF7D8FB401B6428F5D90320B0
S31508006D10AFE1944B5B6813F4803FD6D0914B1B6868
S31508006D2013F4003F03D06368002B00F09F812368AB
S31508006D3013F0020F65D08B4B5B6813F00C0F4ED027
S31508006D40884B5B6803F00C03082B43D02369002BA0
S31508006D5079D00122844B1A60FFF7AEFB0546814BBA
S31508006D601B6813F0020F65D1FFF7A6FB401B02282C
S31508006D70F5D903207DE17B4A136843F48033136019
S31508006D80B5E7B3F5A02F09D0764B1A6822F48032FE
S31508006D901A601A6822F480221A60A8E703F1804371
S31508006DA0A3F53C331A6842F480221A601A6842F442
S31508006DB080321A609BE7FFF77FFB0546694B1B6825
S31508006DC013F4003FB3D0FFF777FB401B6428F5D9CF
S31508006DD003204EE1634B5B6813F4803FB6D1614BE9
S31508006DE01B6813F0020F04D02369012B01D0012080
S31508006DF03FE15C4A136823F0F803616943EAC1037B
S31508006E001360236813F0080F32D0A369002B6ED0E5
S31508006E100122564B1A60FFF74FFB0546514B5B6A3A
S31508006E2013F0020F21D1FFF747FB401B0228F5D9C3
S31508006E3003201EE14B4A136823F0F803616943EA0D
S31508006E40C1031360DDE70022474B1A60FFF734FBE6
S31508006E500546444B1B6813F0020FD2D0FFF72CFBF4
S31508006E60401B0228F5D9032003E10120FFF704FFA0
S31508006E70236813F0040F00F099803A4BDB6913F08E
S31508006E80805F46D1374BDA6942F08052DA61DB69B6
S31508006E9003F080530193019B0125354B1B6813F4BE
S31508006EA0807F38D0E368012B49D0002B4DD103F100
S31508006EB0804303F504331A6A22F001021A621A6A39
S31508006EC022F004021A62E368002B5DD0FFF7F4FA99
S31508006ED00646244B1B6A13F0020F66D1FFF7ECFA3D
S31508006EE0801B41F288339842F3D90320C1E000227F
S31508006EF01E4B1A60FFF7E0FA05461A4B5B6A13F059
S31508006F00020FB5D0FFF7D8FA401B0228F5D903209F
S31508006F10AFE00025C1E7164A136843F4807313608F
S31508006F20FFF7CAFA0646124B1B6813F4807FB9D1DD
S31508006F30FFF7C2FA801B6428F5D9032099E0094AAD
S31508006F40136A43F001031362BDE7052B12D0054B04
S31508006F501A6A22F001021A621A6A22F004021A62F6
S31508006F60B1E700BF001002400000424280044242DE
S31508006F7000700040414B1A6A42F004021A621A6A0B
S31508006F8042F001021A629EE7FFF796FA06463B4B65
S31508006F901B6A13F0020F08D0FFF78EFA801B41F226
S31508006FA088339842F3D9032063E0E5B9E369002BF7
S31508006FB05ED0324A526802F00C02082A5BD0022BD5
S31508006FC017D000222E4B1A60FFF776FA04462B4B91
S31508006FD01B6813F0007F47D0FFF76EFA001B0228E4
S31508006FE0F5D9032045E0254AD36923F08053D361B8
S31508006FF0DCE70022224B1A60FFF75EFA05461F4BB4
S315080070001B6813F0007F06D0FFF756FA401B0228CC
S31508007010F5D903202DE0236AB3F5803F1AD0174926
S315080070204B6823F47413226A606A024313434B6065
S315080070300122134B1A60FFF73FFA04460F4B1B68F1
S3150800704013F0007F0ED1FFF737FA001B0228F5D997
S3150800705003200EE0094A536823F40033A1680B4362
S315080070605360DCE7002004E0002002E0012000E095
S31508007070002002B070BD0120FBE700BF00100240EF
S315080070806000424210B586B0154C94E80F000DF129
S31508007090180E0EE90F00238AADF80430114B5B6811
S315080070A003F00C02082A18D1C3F38342724412F87B
S315080070B0102C13F4803F03D10B4800FB02F00DE0BF
S315080070C0084B5B68C3F34043734413F8143C074802
S315080070D000FB02F0B0FBF3F000E0044806B010BD78
S315080070E0607900080010024000093D0000127A008D
S315080070F0594B1B6803F007038B420CD2564A136898
S3150800710023F007030B431360136803F00703994240
S3150800711001D00120704770B5036813F0020F06D03E
S315080071204E4A536823F0F0038468234353600D46A0
S315080071300446036813F0010F52D04368012B23D08D
S31508007140022B28D0454A126812F0020F00F08280FE
S3150800715042494A6822F0030213434B60FFF7ACF931
S3150800716006466368012B1DD0022B2AD03B4B5B6871
S3150800717013F00C0F34D0FFF79FF9801B41F28833C8
S315080071809842F3D9032070BD344A126812F4003FBE
S31508007190DED1012070BD314A126812F0007FD7D1C6
S315080071A0012070BD2D4B5B6803F00C03042B17D030
S315080071B0FFF782F9801B41F288339842F2D90320FF
S315080071C070BD264B5B6803F00C03082B08D0FFF74D
S315080071D073F9801B41F288339842F2D9032070BDB7
S315080071E01D4B1B6803F007039D420CD21A4A13680D
S315080071F023F007032B431360136803F007039D422C
S3150800720001D0012070BD236813F0040F06D0134A7D
S31508007210536823F4E063E1680B435360236813F073
S31508007220080F07D00D4A536823F46053216943EACF
S31508007230C1035360FFF726FF084B5B68C3F30313CC
S31508007240074AD35CD840074B18600020FFF7F0F8D0
S31508007250002070BD012070BD0020024000100240D1
S315080072609879000808000020014B1868704700BF8D
S315080072700800002008B5FFF7F7FF044B5B68C3F367
S315080072800223034AD35CD84008BD00BF0010024061
S31508007290A879000808B5FFF7E7FF044B5B68C3F356
S315080072A0C223034AD35CD84008BD00BF0010024081
S315080072B0A87900082DE9F04705460268136923F402
S315080072C04053C1680B4313618368026913434269DB
S315080072D013430168CA6822F4B05222F00C02134321
S315080072E0CB600268536923F4407381690B43536189
S315080072F0D0F80080594B984557D0FFF7BBFF00EBF5
S31508007300800000EB80006C68A400B0FBF4F4544FD6
S31508007310A7FB043464092601FFF7ACFF00EB8000E5
S3150800732000EB80006C68A400B0FBF4FAFFF7A2FF3C
S3150800733000EB800000EB80006C68A400B0FBF4F45E
S31508007340A7FB043464094FF0640909FB14A424015B
S315080073503234A7FB0434640904F0F0043444FFF71C
S3150800736089FF00EB800000EB80006E68B600B0FB7A
S31508007370F6F6FFF77FFF00EB800000EB80006B68F6
S315080073809B00B0FBF3F0A7FB0030400909FB10692E
S315080073904FEA091909F13209A7FB0937C7F3431759
S315080073A02744C8F80870BDE8F087FFF773FF00EBBD
S315080073B0800000EB80006C68A400B0FBF4F4284F52
S315080073C0A7FB043464092601FFF764FF00EB80007D
S315080073D000EB80006C68A400B0FBF4FAFFF75AFFD4
S315080073E000EB800000EB80006C68A400B0FBF4F4AE
S315080073F0A7FB043464094FF0640909FB14A42401AB
S315080074003234A7FB0434640904F0F0043444FFF76B
S3150800741041FF00EB800000EB80006E68B600B0FB11
S31508007420F6F6FFF737FF00EB800000EB80006B688D
S315080074309B00B0FBF3F3A7FB03235B0909FB136966
S315080074404FEA091909F13209A7FB0937C7F34317A8
S315080074502744C8F80870BDE8F08700BF0038014027
S315080074601F85EB512DE9F04105460F46164698460D
S31508007470069C2B681B6837EA03030CBF012300230D
S31508007480B3421ED1B4F1FF3FF3D02CB1FFF714F885
S31508007490A0EB08008442ECD22A68D36823F4D073A0
S315080074A0D3602A68536923F001035361202385F8C2
S315080074B0393085F83A30002385F838300320BDE89E
S315080074C0F0810020BDE8F081704758B310B5044636
S315080074D090F839300BB3242384F839302268D368FE
S315080074E023F40053D3602046FFF7E4FE22681369AD
S315080074F023F4904313612268536923F02A035361E6
S315080075002268D36843F40053D3600020E063202345
S3150800751084F8393084F83A3010BD80F83830FFF7EF
S31508007520D3FFD8E7012070472DE9F04182B01E4607
S3150800753090F83A30DBB2202B03D0022002B0BDE827
S31508007540F08104460D469046002958D0002A58D0A6
S3150800755090F83830012B01D10220EFE7012380F89B
S3150800756038300023C363222380F83A30FEF7A4FF9D
S315080075700746A4F82C80A4F82E801DE000963B460A
S31508007580002220212046FFF76DFF00283BD1236902
S3150800759033B923685B68C3F3080325F8023B0BE09D
S315080075A023685B68DBB225F8013B05E023685B6866
S315080075B003F07F032B700135E38D9BB2C3B1E38DD6
S315080075C09BB2013B9BB2E385A368B3F5805FD5D038
S315080075D000963B46002220212046FFF743FFA0B92C
S315080075E02369002BE2D123685B682B700135E3E73A
S315080075F0202384F83A30002084F838009EE70120DA
S315080076009CE701209AE7032098E7032096E7000005
S315080076100F4B1A6842F001021A6059680D4A0A406F
S315080076205A601A6822F0847222F480321A601A6844
S3150800763022F480221A605A6822F4FE025A604FF435
S315080076401F029A604FF00062034B9A60704700BFB2
S31508007650001002400000FFF800ED00E0014B024A6E
S315080076609A60704700ED00E00060000800B591B030
S31508007670012206924FF480330793002108910A925B
S3150800768002220D920E934FF4E0130F9306A8FFF70C
S3150800769009FB00B1FEE70F230193022102910023A3
S315080076A003934FF480620492059301A8FFF720FD27
S315080076B000B1FEE711B05DF804FB08B5FFF7CEFF91
S315080076C0FEF7DCFEFFF7D2FF00F0FAF8FEF77CFEC5
S315080076D008BD08B5FFF7F1FFFEF7EAFDFEF77EFEE7
S315080076E0FEF76CFEFAE700002DE9F0418CB05B4B23
S315080076F09A6942F001029A619A6902F001020192BE
S31508007700019ADA6942F08052DA61DA6902F0805247
S315080077100292029A9A6942F004029A619A6902F000
S3150800772004020392039A9A6942F008029A619A69D6
S3150800773002F008020492049A9A6942F010029A61C9
S315080077409A6902F010020592059ADA6942F4003243
S31508007750DA61DA6902F400320692069ADA6942F0C8
S315080077600072DA61DB6903F000730793079B032055
S31508007770FFF716F9002211466FF00B00FFF722F902
S31508007780002211466FF00A00FFF71CF90022114685
S315080077906FF00900FFF716F9002211466FF0040092
S315080077A0FFF710F9002211466FF00300FFF70AF9F8
S315080077B0002211466FF00100FFF704F90022114676
S315080077C04FF0FF30FFF7FEF84FF4805708974FF059
S315080077D00108CDF8248000240A9402250B95204E32
S315080077E008A93046FFF74CF9424639463046FFF7B6
S315080077F03DFA04230893099503260B9607F180475B
S3150800780007F5784708A93846FFF73AF90823089391
S3150800781009940A9408A93846FFF732F94FF4807399
S31508007820089309940A940F4C08A92046FFF728F9EB
S315080078304FF40073089309950B9608A92046FFF79D
S315080078401FF9094A536823F4C04343F0E06343F43D
S31508007850804353600CB0BDE8F08100BF00100240C1
S3150800786000100140000C014000000140DFF834D050
S31508007870002103E00C4B5B58435004310B480C4B7A
S3150800788042189A42F6D30B4A02E0002342F8043B18
S31508007890094B9A42F9D3FFF7BBFE00F031F8FFF720
S315080078A018FF704700500020B87900080000002033
S315080078B00C0000200C00002024010020FEE7000038
S315080078C008B5FFF7D1FC084BA3FB00308009FFF78A
S315080078D0ABF80420FFF7BEF8002211464FF0FF3040
S315080078E0FFF770F808BD00BFD34D621008B5FEF764
S315080078F0E3FD08BD08B5FEF7D3FDFFF7BCF808BDE4
S3150800790070B500250C4E0D4CA41BA410A54209D138
S3150800791000F01AF800250A4E0A4CA41BA410A5422A
S3150800792005D170BD56F8253098470135EEE756F86B
S31508007930253098470135F2E7B0790008B079000894
S31508007940B0790008B4790008F8B500BFF8BC08BCDF
S315080079509E467047F8B500BFF8BC08BC9E467047FF
S3150800796002030405060708090A0B0C0D0E0F101072
S3150800797001020000050206020603070308030903BD
S3150800798009040A040B040C040C050D050E050F0565
S315080079900F0610061007100800000000000000007F
S315080079A00102030406070809000000000102030497
S309080079B03561000827
S309080079B41161000847
S311080079B8010000001000000000A24A04B4
S7050800786D0D
